:100000000C9454000C9466000C9466000C946600EA
:100010000C9466000C94EA090C9466000C9466003B
:100020000C9466000C9466000C9466000C946600B8
:100030000C9466000C9466000C9466000C946600A8
:100040000C94F8080C9466000C9466000C942E092D
:100050000C9466000C9466000C9466000C94A8093D
:100060000C9466000C9466000C9466000C94660078
:10007000C0000000C0000000000000000000000000
:100080000000000000000000E0000000FFE00000B1
:1000900004B6E704B6D304B6C704B6C30290070398
:1000A000AC8103AC8002900011241FBECFEFD4E0DE
:1000B000DEBFCDBF24E0A0E0B1E001C01D92AD36AF
:1000C000B207E1F70E9482080C94570A0C940000D2
:1000D0001F93CF93DF931F92CDB7DEB7182FBC9A33
:1000E00069830E948C02959882E00E949102812F80
:1000F0000E9491026981862F0E949102959A1DB8F3
:10010000BC980F90DF91CF911F910895CF93C82F86
:10011000BC9A0E948C02959883E00E9491028C2FD9
:100120000E9491028FEF0E949102959A1DB8BC988F
:10013000CF9108951F93CF93DF9300D0CDB7DEB753
:10014000182FBC9A4A8369830E948C02959885E097
:100150000E949102812F0E9491026981862F0E9444
:1001600091024A81842F0E949102959A1DB8BC98F1
:100170000F900F90DF91CF911F910895CF93DF9350
:100180001F92CDB7DEB7BC9A89830E948C029598E6
:1001900089810E9491028FEF0E949102959A1DB869
:1001A000BC980F90DF91CF910895EF92FF920F933B
:1001B0001F93CF93DF93E82E87E08E1510F480E035
:1001C00062C010926C04959A8D9AC798C598C6988B
:1001D000BF9ABD9ABE98BC9A0E948C02959880ECFA
:1001E0000E94910283E397E00197F1F7959A8FEFD0
:1001F00097E40197F1F700C00000959882E00E9413
:10020000910288E20E94910293E0E99E800111240C
:10021000C0E0D0E0F12C00571F4FF801EC0FFD1F9C
:1002200084910E9491022196C330D105B1F783E0F9
:100230000E949102959A1DB8BC9860E08DE00E94E2
:100240006800A298AA9AA398A498AB9AAC9A6FE077
:100250008CE00E94680089E20E948600D82FF70196
:10026000EE0FFF1FEE0DFF1DEF56FF4FC49160E034
:100270008FE00E946800DC13A2CF8EE00E9486000F
:10028000807ED9F781E0DF91CF911F910F91FF9090
:10029000EF90089583B382FB882780F991E0892746
:1002A000089580EA0E94BE00982F947581E009F0BD
:1002B00080E00895CF92DF92FF920F931F93CF9328
:1002C000DF931F92CDB7DEB76C0180916C04882359
:1002D00031F09C9904C010926C0484E910C09B9981
:1002E00008C010926C049C9909C081E080936C0452
:1002F00005C09C9BF0CF10926C0412C080E9BC9AA0
:1003000089830E948C02959889810E949102C6017E
:100310000E945802182F80FF05C0959A1DB8BC98FE
:1003200080E01FC08FEF0E94910216951170F601B8
:10033000928110FB90F992838F70F82E838300E0F6
:1003400010E00F1550F48FEF0E949102F601E00FBC
:10035000F11F84830F5F1F4FF4CF959A1DB8BC988F
:1003600081E00F90DF91CF911F910F91FF90DF906F
:10037000CF900895FF920F931F93CF93DF93EC01DB
:1003800080EA0E94BE0082FD34C0BC9A0E948C02AA
:10039000959880E40E949102CE010E944002FB8069
:1003A0008F2D8F70F82E8A8180FF05C08F2D80647D
:1003B0000E94910210C08F2D0E94910200E010E077
:1003C0000F1548F4FE01E00FF11F84810E94910295
:1003D0000F5F1F4FF5CF959A82E08A95F1F700C025
:1003E000959881E80E949102959A1DB8BC9881E089
:1003F00001C080E0DF91CF911F910F91FF90089590
:100400000F931F93CF93DF93EC0140E860EE8FE0F2
:100410000E949A008EE00E948600807E8038D1F78C
:1004200064E080E60E94680060E080E70E94680067
:1004300010E0BC9A0E948C02959882E00E94910282
:10044000812F0E94910200E0103211F4083048F42C
:100450002196FE01319784910E9491020F5F0C302A
:1004600099F7959A1DB8BC98105F103311F740E0CA
:1004700060EE8FE0DF91CF911F910F910C949A0065
:10048000FC012081318183E0369527958A95E1F73B
:100490002FB980818295880F807E779BFECF9FB198
:1004A0000E94910280E00E94910280E00C949102EF
:1004B0001F93CF93DF93EC018FEF0E949102182FCF
:1004C0008FEF0E949102982F8FEF93FF07C00E9439
:1004D00091028FEF0E94910281E01AC08FB988E0EB
:1004E000189F9001112439832883779BFECF8FB109
:1004F0008FEF8FB98881292F229526952770822B1F
:100500008883779BFECF8FB1892F807194FD82E025
:10051000DF91CF911F91089581E58DB981E08EB96A
:1005200008958FB9779BFECF8FB10895CF938091B7
:100530001501882341F090911301911104C090910D
:1005400014019923A1F190916804911114C08111B3
:1005500012C08091000181110EC080916704811149
:100560000AC08091590390915A0321E0892B09F028
:1005700020E0822F01C080E095B7906295BF9BB7C5
:1005800090619BBFC82FC17080FF02C08DE083BF08
:100590000E944A01811101C08895CC2311F08BE0A3
:1005A00083BF8BB78F7E8BBF85B78F7D85BFCF9184
:1005B00008951F93CF93DF9300D0CDB7DEB76115B9
:1005C000710509F468C0F8942091590330915A03D9
:1005D0003A832983789429813A81260F371F29315C
:1005E000314008F05AC020915D0330915E03FC0158
:1005F000AC01460F571FE417F50781F0C9010196BA
:1006000011912F5B3D4FD9011C938831B1E09B07BD
:1006100010F49C01F0CF20E030E0EDCF30935E038A
:1006200020935D03F8942091590330915A038091EF
:10063000590390915A03860F971F90935A03809302
:100640005903232B11F0789426C080915B0390917D
:100650005C039C012F5F3F4F30935C0320935B034F
:10066000FC01EF5BFD4F80818CB980915903909123
:100670005A03019790935A038093590380915B0327
:1006800090915C038831914020F010925C031092AD
:100690005B03569AD8CF81E001C080E00F900F90A5
:1006A000DF91CF911F910895CF93DF93209167043D
:1006B000223069F4C0916504D0916604AE016FE503
:1006C00073E00E94210A10926704CE0102C080E00C
:1006D00090E0DF91CF91089528E088E190E00FB697
:1006E000F894A89581BD0FBE21BD85B7806285BFF6
:1006F000889585B78F7D85BFF8CF80916804882362
:1007000031F080916904833310F010926804809175
:100710006804882311F039980DC0809167048823FC
:1007200011F0399A01C039988091590390915A0378
:10073000892B11F0389A01C03898809131018111CC
:1007400002C0B49B02C03A9808953A9A0895FC01F9
:10075000680F791F80E0E617F70719F09191890F6C
:10076000FACF089580E090E00E942A0AAC014095FB
:100770005095452F55279C0133274217530709F001
:1007800081E08093310182E090E00E942A0AAC016E
:1007900040955095452F55279C0133274217530705
:1007A00019F01092300102C08093300184E090E093
:1007B0000E942A0AAC0140955095452F55279C016F
:1007C00033274217530719F010922F0102C080936C
:1007D0002F0186E090E00E942A0AAC0140955095D6
:1007E000452F55279C0133274217530719F01092C4
:1007F0002E0102C080932E0180912E018BBB0895A3
:1008000080913101882331F0893041F081E080937B
:10081000320102C01092320186E004C081E0809370
:10082000320183E010921501109200019091320183
:100830009923A1F0949A0E94D50081110BC0389899
:10084000399AF89485B7806285BF889585B78F7D82
:1008500085BFF8CF80E790E00C940002949808954B
:100860001F93CF93DF93EC0110916904CE010E9496
:10087000BA01811109C00E947D0380916904811B26
:100880008A31A0F380E001C081E0DF91CF911F9118
:1008900008958530910529F580913D01813809F051
:1008A0000BC180913E01811107C180913F018111EF
:1008B00003C18091400190E0BC0160957095762F56
:1008C0006627682B792B80E090E00E94300A0E9416
:1008D000B2030E9400048091310180958093400111
:1008E0007DC0069709F0E8C080913D01823809F08B
:1008F000E3C080913E01813F09F0DEC080913F015D
:10090000813F09F0D9C080914001982F9F77A9F4C9
:1009100087FD10C08091410190E0BC016095709509
:10092000762F6627682B792B82E090E00E94300AB0
:100930000E94B20380913001A4C09130A9F487FDD8
:1009400010C08091410190E0BC0160957095762FB8
:100950006627682B792B84E090E00E94300A0E9481
:10096000B20380912F018DC09230B9F487FD12C07F
:100970008091410190E0BC0160957095762F6627CB
:10098000682B792B80E090E00E94300A0E94B2032D
:100990000E9400048091310174C09330A9F487FD56
:1009A00010C08091410190E0BC0160957095762F58
:1009B0006627682B792B86E090E00E94300A0E941F
:1009C000B20380912E015DC0843899F48091410179
:1009D000843809F06FC081E880933D0164E070E0E5
:1009E0008DE391E00E94A7038093410165E070E0F0
:1009F00054C0853831F480914101853809F05AC0DE
:100A0000EACF8B3F31F4809141018B3F09F052C016
:100A1000E2CF8C3F39F4809141018C3F09F04AC00C
:100A200080E82FC08D3FE1F4809141018D3F09F0B6
:100A300041C085E880933D011092410181E080939F
:100A40004201109243018093440168E070E08DE31D
:100A500091E00E94A7038093450169E070E01DC00A
:100A60008E3F01F5809141018E3F21F596B392951D
:100A7000917080913101882311F080E801C080E0FD
:100A8000892B8093410165E070E08DE391E00E9445
:100A9000A7038093420166E070E08DE391E00E943D
:100AA000D90208C08F3F31F4809141018F3F11F48A
:100AB0000E946C0381E0089580E00895EF92FF9218
:100AC0000F931F93CF93DF93082F809132018823D8
:100AD00009F455C180911501811113C08DE391E096
:100AE0000E945403009769F00E944904811147C194
:100AF00081E080931501109213011092120110925F
:100B0000110180911501882309F439C1F0903D014C
:100B10002F2D2F73F22E29F4F0904001E1E4F1E043
:100B200002C0E0E4F1E040913E0110913F01C0912C
:100B30001101D0911201209709F054C0812F90E04B
:100B4000A6E02CE0AF15F0F0A2E2B1E0ED011992C1
:100B50002A95E9F79660909323018093220188E01B
:100B60008093250140932601F09227014F2D50E0FC
:100B7000BF0188E291E00E94210A82E291E00E9496
:100B80003004D2C0A2E2B1E0ED0119922A95E9F752
:100B90009660909323018093220188E08093250141
:100BA0004093260180E180932701F092280185E09F
:100BB000A9E2B1E001900D928A95E1F785E090E01D
:100BC000909312018093110182E291E00E9430041F
:100BD00081E08093140180931001809169048093D7
:100BE0000C01CDC080911401882309F43FC000237B
:100BF00079F12091160130911701B901662761152D
:100C0000764031F580911901843010F1332750E09E
:100C100024173507E9F480911A01811319C08091D6
:100C20001B01982F907F903399F48F7039F08130A9
:100C300039F48091690480930C0102C01092140170
:100C400080911C0180930F0180911D0180930E0102
:100C500080911401882309F492C0809169049091D5
:100C60000C01891B853608F48AC05EC0909113017F
:100C70009923E1F030910D0180910E01913031F412
:100C800090916A04931B891778F079C020916904C8
:100C9000231B30E090E009966AE070E00E94F909B9
:100CA000621773070CF06BC0109213018CE022E204
:100CB00031E0D9011D928A95E9F7812F90E0966085
:100CC000909323018093220188E080932501409333
:100CD0002601E09010018E2D8F7080628093270195
:100CE0000F2D0C1B073008F006E010E0BF016C0F61
:100CF0007D1FA80188E291E00E94210AC00FD11F48
:100D0000D0931201C0931101E394E092100182E2AA
:100D100091E00E9430044F2D50E08091110190919C
:100D200012018417950718F01092150128C010922F
:100D3000140180910F01882359F0813031F48093A0
:100D400014019091690490930C01815080930F01DC
:100D500080911401811113C080910E01882379F0D4
:100D6000843630F481E08093130180916A0405C0D9
:100D700082E0809313018091690480930D01DF91DB
:100D8000CF911F910F91FF90EF9008959F92AF9296
:100D9000BF92CF92DF92EF92FF920F931F93CF9368
:100DA000DF9300D01F92CDB7DEB790913201992327
:100DB00009F499C1882309F489C1809116019091A1
:100DC00017019C0122272115364009F038C1E09116
:100DD0001901E23008F433C120911B01322F329502
:100DE0003F703130A1F120F0323009F4AFC027C19B
:100DF00030911A01F0E03197422F50E04E175F0713
:100E00000CF01DC1922F9068909333013093340100
:100E1000809335016CE171E086E391E02B830E94C1
:100E2000210A2B8103E0020F10E0B80183E391E077
:100E30000E94A703F801ED5CFE4F80832B812C5F9D
:100E4000622F70E083E391E00E94D902F8C03091F4
:100E500000013111F4C0E83008F4F1C080930901B9
:100E600070911A01709308012F7030E0322F222701
:100E700040911C01240F311D309302012093010188
:100E80002F3F310521F018F010920001D8C0203416
:100E9000310518F041E451E002C040E451E05093C4
:100EA0000B0140930A01A0910A01B0910B0195E05A
:100EB000EDE1F1E001900D929A95E1F745E050E007
:100EC000509304014093030191E0909307012CE0BB
:100ED000E2E2F1E0DF011D922A95E9F7272F30E0E9
:100EE0003660309323012093220128E020932501CE
:100EF0008093260180E380932701809130018093C5
:100F0000280120912F0120932901809306019093BD
:100F1000000108E111E0F8948091590390915A037F
:100F20009A838983789489819A819801281B390B47
:100F3000809101019091020105962817390718F454
:100F40000E949602E8CF82E291E073C030910001E6
:100F5000332309F474C0B09009014B2D50E0992758
:100F60004817590709F06BC0A090080180911A0139
:100F7000A81265C09090070129252F7009F05FC065
:100F8000C0900101D0900201E0900301F0900401B3
:100F900086010E191F090730110510F006E010E058
:100FA0002E2F30E0225031092017310708F447C0B6
:100FB00080910A0190910B01A8016CE171E08E0D06
:100FC0009F1D0E94210A0E0D1F1D10930401009306
:100FD000030193949092070180910601882359F1AF
:100FE0000C151D0540F5815080930601811123C029
:100FF0008CE0E2E2F1E0DF011D928A95E9F78A2DAB
:1010000090E09660909323018093220188E0809382
:101010002501B092260180E3809327018091300161
:101020008093280190912F019093290180930601CC
:10103000CF010E9430048091690480930501809162
:101040000001882309F44FC06091010170910201F1
:1010500080910301909104018617970708F443C01B
:1010600080910901909108016034710568F020E8D1
:1010700020933D0190933E0180933F016093400196
:101080008B010C5F1F4F0BC0262F206820933D0162
:1010900090933E0180933F018B010D5F1F4FB8017C
:1010A0008DE391E00E94A703F801E35CFE4F80838B
:1010B000B8016F5F7F4F8DE391E00E94D9028111EB
:1010C00010C080916904809305010DC080910001DA
:1010D000882349F08091690490910501891B853628
:1010E00010F0109200010F900F900F90DF91CF91B0
:1010F0001F910F91FF90EF90DF90CF90BF90AF9036
:101100009F90089510926B0410926A0410926904E3
:1011100081E0809368041092670410926604109234
:1011200065041092640410925E0310925D031092A5
:101130005C0310925B0310925A03109259031092B1
:10114000150110920001479A80916C008460809391
:101150006C008FE78ABB1BBA80E181BB949887E063
:1011600086B93998389A3A9A8BE083BF82E781BF73
:1011700089B7816089BF93E099B988E18AB9579AA4
:1011800086E880BD90B998E091B98CBF85B78F7E15
:1011900085BF84B78F7D84BF86B78F7786BF7894ED
:1011A0000E94B2030E94000480913201882399F0CA
:1011B0000E944A01882339F086E191E00E945A0199
:1011C000C1E0811101C0C0E08C2F0E94C6068C2FA7
:1011D0000E945E0508C08DE391E00E9454030097D1
:1011E00011F00E9449040E947D030E949602DCCF08
:1011F0001F920F920FB60F9211248F9380916A0461
:101200008F5F80936A0480916B048F5F80936B047F
:1012100080916B048A3038F010926B0480916904DD
:101220008F5F8093690480916404882389F08091A2
:10123000640481508093640480916704813011F0CC
:10124000833031F480916404811102C010926704EC
:101250008F910F900FBE0F901F9018951F920F92B5
:101260000FB60F9211242F933F934F935F938F9359
:101270009F93EF93FF934CB183E08093640480913C
:101280006704882319F08130C1F055C010926604BC
:101290001092650480916504909166049C012F5F13
:1012A0003F4F3093660420936504FC01E15AFC4FE4
:1012B00040834093630481E038C08091650490913D
:1012C00066048430914078F48091650490916604BE
:1012D0009C012F5F3F4F3093660420936504FC010F
:1012E000E15AFC4F408380916504909166045091CF
:1012F00063040497E8F080915F038F7390E0009798
:1013000029F48091620390E0059601C00496209133
:101310006504309166042817390750F0541711F00E
:1013200083E003C01092640482E08093670403C0EA
:10133000450F40936304FF91EF919F918F915F91CF
:101340004F913F912F910F900FBE0F901F901895C6
:101350001F920F920FB60F9211242F933F938F93EA
:101360009F93EF93FF938091590390915A03892B98
:1013700011F4569824C080915B0390915C039C010A
:101380002F5F3F4F30935C0320935B03FC01EF5BC7
:10139000FD4F80818CB98091590390915A03019738
:1013A00090935A038093590380915B0390915C035F
:1013B0008831914020F010925C0310925B03FF9102
:1013C000EF919F918F913F912F910F900FBE0F90B2
:1013D0001F9018951F920F920FB60F9211248F93A2
:1013E00085B78F7D85BF8F910F900FBE0F901F9097
:1013F000189597FB072E16F4009407D077FD09D0B7
:101400000E940D0A07FC05D03EF4909581959F4FF0
:101410000895709561957F4F0895AA1BBB1B51E1FC
:1014200007C0AA1FBB1FA617B70710F0A61BB70B54
:10143000881F991F5A95A9F780959095BC01CD01F9
:101440000895FB01DC0102C001900D924150504013
:10145000D8F70895A8E1B0E042E050E00C94380AD3
:101460000196272F0E94470A0C94460ADC01CB0103
:10147000FC01E199FECF06C0FFBBEEBBE09A3196BE
:101480000DB20D9241505040B8F70895262FE199C2
:10149000FECF9FBB8EBBE09A01970DB2021631F0D2
:1014A0002DBB0FB6F894E29AE19A0FBE0895F89416
:0214B000FFCF6C
:00000001FF
